:030000000219FDE5
:03000B000200AA46
:03002B000201656A
:03005B000202FBA3
:030073000202E1A5
:1000800002030406080C10182030406080040608A3
:100090000C10182030406080A0C000070F1F3F0DDB
:1000A0000D0403060D0503030202C2AFC0D0C0E079
:1000B000206217E5256002E473E525F4F58A758B67
:1000C00000D262D0E0D0D0D2AF3285268AC262E5BB
:1000D00026F46035306803207210758B00D0E0D0B4
:1000E000D0D292D291D290D2AF32D292D291D2903B
:1000F000206E0C206609740AD5E0FDE57E429075FD
:100100008B00D0E0D0D0D2AF32758A00C28DD262DF
:1001100001FF01B9306805206602C29201B930685A
:1001200005206602C29101B9306805206602C290BE
:1001300001B9C29530680A2066077408D5E0FDC28F
:100140009201B9C29430680A2066077408D5E0FDB0
:10015000C29101B9C29330680A2066077408D5E0DD
:10016000FDC29001B9C2AFC2AD53E6EFC0D0C0E04E
:10017000D2D3D2AFC2CEE52A6007207449152A2116
:10018000C67800790020742EE580307E01F430E7D7
:100190000278FF53DACF207E0343DA20307E034318
:1001A000DA10C2D8C271E580307E01F430E70279FE
:1001B000FFC3E89970CB306103752A402074037542
:1001C0002A40885FD27020740DE52B6004152B2126
:1001D000D643DA01C2D820700221E9A85F2061026B
:1001E000C27020740221E788227882B60403852237
:1001F00024C3E52594404002D26420CF0AD0E0D049
:10020000D043E610D2AD32C2CF053A7802E52A607B
:1002100005307402152AC3E55F940140057562003C
:100220004133756300756C00E5622401F56250038B
:100230007562FF7982B7020D306D1DC3E5229432DD
:100240004016854D227982B7030E306D0BC3E5222F
:1002500094324004798E8722C3E5239522600840BA
:1002600004152341670523D8CA056CE56C70021597
:100270006CD56D63756D017805C3E56C956E40575F
:10028000C3E56C956F50087801756D0302029BC33E
:10029000E56C957050057801756D01C3E565952491
:1002A000401E7982B7040241CC206D14852465E597
:1002B0006C046003856E6C756D0175233C0202D77A
:1002C000E5652850057565FF41CCF565E565047069
:1002D000067563FF756CFFD0E0D0D043E610D2AD59
:1002E00032C2AFC0D053E67FC2607591008556948C
:1002F000855795759104D0D0D2AF32C2AF53E6EF97
:10030000C2ADC0D0C0E0C0F0D2D3D2AFA8FBA9FC30
:10031000C2D8307102616253DACF207E0343DA1013
:10032000307E0343DA20D271E580307E01F420E78D
:1003300002613988278928A14153DACF207E0343FF
:10034000DA20307E0343DA10C2D8C271307402A1C1
:100350002D7800E580307E01F430E702A12D885F22
:10036000A11553DACF207E0343DA20307E0343DA2F
:1003700010C271206102813B53DACF207E0343DA41
:1003800010307E0343DA20C2D8D271885A895BC309
:10039000E89558F8E99559F97B007E087A00C3E89A
:1003A000948CE994005005755E00812D882178A217
:1003B000E6A8216055C3E894C8E994005008E4D247
:1003C000E4FB7A0A8108C3E89468E994015008E4E0
:1003D000D2E3FB7A0F8108C3E894D0E99402500875
:1003E000E4D2E2FB7A1E8108C3E894A0E9940550A8
:1003F00008E4D2E1FB7A3C8108C3E89498E99408C8
:100400005008E4D2E0FB7A787E00C3E8955CFCE912
:10041000955DFD30E70AECF42401FCEDF43400FDB9
:10042000755E00C3EC9AED9E5003755E01885C8991
:100430005D855A58855B597802A115C3E89527F860
:10044000E99528F9307C0281F9307B0281F9307A14
:100450000281F2207502815EE9FDE8FC817DE9C33D
:1004600013F9E813F830790281F2E9C313F9E813BC
:0D047000F830780281F2E9C313FDE813FCB7
:10047D00206126C3EC941CED940240028194ED7032
:10048D0018C3EC94C850120529C3E529940A5002EB
:10049D00A12D755F00D270A12DE52960021529747B
:1004AD0000207F037896E624FAFEE43400FFC3ECC7
:1004BD009EFCED9FFD50067800790081F9C3EC9408
:1004CD00FFED9400400678FF790081F9EC8575F019
:1004DD00A4C5F0A2F733F87900400302051578FFA3
:1004ED007900020515E9C313F9E813F8307C0EE91C
:1004FD00600278FFC3E81338F8E43400F9C3E894D8
:10050D00FFE99400400278FF885FD270206102A15C
:10051D002D741FF4552F4BF52FC274EB7002D2744E
:10052D00752A40307403752A0A306102A141207486
:10053D000353DAFE207403752B20D0F0D0E0D0D019
:10054D00D2AD43E6103279010205717903020571CE
:10055D00790A020571791E020571796402057179B6
:10056D00C80205717817E4D5E0FDD8FAD9F6227ADC
:10057D00147B780205987A107B8C0205987A0D7B96
:10058D00B40205987A0B7BC80205987902B27DE416
:10059D00C294D5E0FDC291D5E0FDD291D5E0FDD25A
:1005AD0094D5E0FDC292E576D5E0FDD2927496D554
:1005BD00E0FDD9D9EAF8D5E0FDD8FBDBCEC2942217
:1005CD00C37C007D0075F00005F0EA33FAEB33FBD8
:1005DD0050F6EB13FBEA13FAC3E9FFE8FEE89AF8CD
:1005ED00E99BF95004EFF9EEF8B3EC33FCED33FD74
:1005FD00D5F0DFEDF9ECF822E889F08A20D2D4F8B5
:10060D00A9F07B0030F70B7BFFF42401F8E9F434FB
:10061D0000F9E88520F0A4ADF0F8E98520F0A4AF4D
:10062D00F0FEED2EF974003FFA7C04C3EA13FAE9EB
:10063D0013F9E813F8DCF48BF030F70AE8F4240131
:10064D00F8E9F43400F9E889F0C2D4F8A9F0227879
:10065D0082B604030206FBC3E55F9419401EE52D27
:10066D0054067018206D3678057994E71460077874
:10067D000A1460027812C3E54198401F306D098558
:10068D006765756CFF756D01852224E4F545F546AA
:10069D00F547F548F549C26D0206FBD26D7994E731
:1006AD00147013E523F43333F913F8E9540104F905
:1006BD00E854FE0206EFE714147014E523F4333307
:1006CD0033F913F8E9540304F9E854FC0206F7E58D
:1006DD0023F433333333F913F8E954070404F9E8F9
:1006ED0054F8C39440F8E99400F98845894622C32B
:1006FD00E54113F9E54013F8C3E54598F8E546994A
:10070D00F9500CC3E89480E994FF4016020733C3F7
:10071D00E8947FE994005003020733787F79000253
:10072D000733788079FF884A894B22E54A2547F8B7
:10073D00E54B3548F9854B20E4300701F43549FA8E
:10074D0030E709C3EA94F04015020771C3EA940F2C
:10075D00500302077178FF79FF7A0F020771780055
:10076D0079007AF0C3E5249564500AC37401952489
:10077D00500B02078FE54B20E70E02078FE54B303C
:10078D00E706884789488A492278A4E6FAC3E54AEC
:10079D0033F8E54B33F9D105E930E70BC3E8948025
:1007AD00E994FF4013E1C9C3E8947FE99400500236
:1007BD00E1C9787F7900E1C9788079FFE820E715F4
:1007CD00C3E52398F84009C3E8940140030207F0FC
:1007DD0078010207F0E8F424012523F8400302070D
:1007ED00F078FF884C2278A5E6FAA848A949D105EA
:1007FD00E930E70CC3E89401E994FF4016020824A0
:10080D00C3E894FFE99400500302082478FF7900AF
:10081D00020824780179FFE920E715C3E54C98F823
:10082D004009C3E89401400302084B780102084BCC
:10083D00E8F42401254CF8400302084B78FF882486
:10084D002278FFC26420693D206A12D264C3E5415B
:10085D00940A4009C3E52594405002C26479A1E78A
:0F086D006023E541601F74FF8541F0848539F0F9
:10087C00306A0375F005A4F8C5F0600278FFC3E890
:10088C0095675002A867886622C3E5409440E5410D
:10089C009401E56650031401A6046002F566227803
:1008AC0083E6F520120F4575E89012055375E89014
:1008BC00E5E820ECFBA8BDA9BE120FDF75715575DC
:1008CC007200C3740013FD7455606613FC74552CD0
:1008DC00FC74003DFDECFAEDFBC3E89AE99B401477
:1008EC00E5712455F571E5723400F572EA2CFAEBDA
:1008FC003DFB80E5AE71AF72C3E57213F9E5711380
:10090C00F8C3E913F9E813F87A03C3E913F9E81308
:10091C00F8DAF7AA201A70097571007572000209CD
:10092C003D1AEA6008EE28FEEF39FFDAF88E718F77
:10093C00722275E890227883E6FFE5E820ECF7A8B0
:10094C00BDA9BE0573C3E57394084052757300E9E5
:10095C00FA79A0E76044EA7007E574601B02097835
:10096C00C3E895746010E5745006600C1402098499
:10097C000460F9020984E574F574C3946D401B7529
:10098C0064C0C394044013756480C39404400B7515
:10099C006440C39404400375640075BB0622EFC326
:1009AC009401601F7455601BC3E894FFE9940350D5
:1009BC0012C3E89571E995725009E564600C1564F1
:1009CC000209D6E564F460020564A864C3E52498C2
:1009DC005002A824C3E89565400AA865E565F46053
:1009EC000385656488258826E573B4070375BB10F9
:1009FC0022743279A687F0A4C5F0A2F733F8C3E8C5
:100A0C0095644002A86488228824882588268867F3
:100A1C00227540007541F022C2AF75C820A8CCA940
:100A2C00CDAA3A30CF010A75C824D2AFAB3BAC3C4F
:100A3C00883B893CC3E89BF8E99C206908F930673E
:100A4C000261394196AD3D8A3DF9EA9DFA60047820
:100A5C00FF79FFAE3EAF3F8B3E8C3FC3EC9FFCC398
:100A6C00E99CF542A83BA93CC3E89EF8E99FF9C371
:100A7C00E54113FBE54013FAE82AF540E93BF54163
:100A8C0050067540FF7541FF41E0AA40AB41AC40B8
:100A9C00AD417E047F02C3EB940440021E1FC3EBE6
:100AAC00940840021E1FC3ED13FDEC13FCDEF7C3CC
:100ABC00EA9CFAEB9DFBEF6009C3E913F9E813F824
:100ACC00DFF7EA28FAEB39FB8A408B4150067BFFB3
:100ADC008B408B41C3EB94025002D2673069047F88
:100AEC0003610B7892E6FFC3E537948240110FC384
:100AFC00E53794A040010FC3EF940640027F057EBA
:100B0C0005E541C4540FF9E541C454F0F8E540C47F
:100B1C00540F28F8C3E89EFAE99400FB4009C3EA95
:100B2C009402EB940050047A02E4FB6185AA40AB7A
:100B3C0041EBC4FEEAC4540F4EFCC3EA9CFAEB949E
:100B4C0000FBC3E813C313F8EA28FAEB3400FB8A62
:100B5C00408B41C3EB94024002C2677805EBC4FEA4
:100B6C007B00EAC4540F4EFAC3EA98FA4005C394CA
:100B7C000250027A027892E6FF306002618585525B
:100B8C0056855357D26043E680C3E49AF8E49BF948
:100B9C00306702811FE8FAE9FBD3E913FDE813FC87
:100BAC0088528953C3EF94036038EF20E00DE82C92
:100BBC00F8E93DF9ECFAEDFB020BDAE828F8E93933
:100BCC00F9C3E82402F8E93400F97AFE7BFFC3EF9D
:100BDC009403400E8A548B55884E894F8C508D51FE
:100BEC008153885489558A4E8B4F8C508D51306966
:100BFC0020C3E53394034019E542A2E713F8E55509
:100C0C00F4240138400B20E7087554FFF42401F557
:100C1C00558153E8FAD3E813FC8852C3EF94036070
:100C2C0020EF20E007E82CF8ECFA813FE8282402BA
:100C3C00F87AFEC3EF940340088A54884E8C508196
:100C4C005388548A4E8C50E56BC3335002646BF559
:100C5C006B306002815D753402D26043E680E52D15
:0F0C6C0054066026A840A941C3E913F9E813F81C
:100C7B00C2AF53E67F759100C3E498F594E499F500
:100C8B0095759104D26043E680D2AF22D26575444C
:100C9B0000752000306B03752040020CB6D26575D1
:100CAB004400752040306B03752000D2AF780120D3
:100CBB006722E52D54066002C265C3E541940540E9
:100CCB0013780294054008780394054002780630A7
:100CDB006902780A206019E544601530690AC3E59A
:100CEB003394034003D53406D2AFD26CA1889165FF
:100CFB00D2AF0000C2AF206726E541C3FB940F4083
:100D0B00027B0FEB240530730123306A0274282019
:100D1B00620123F93069027982E58BC39940B505ED
:100D2B0044E59BF45440B52002A17230690A08C314
:100D3B00E8940A40010881DF20650281B6C2655341
:100D4B00E67F7591003067107594007595FE75916F
:100D5B0004D26043E68081B6AE40AF41C3E49EF55A
:100D6B0094E49FF595A159C3E5339402500281B6E3
:100D7B0030650281B6D802A18681DFC26C53E67F53
:100D8B00759100855494855595759104854E5685BE
:100D9B004F57D26043E680D2AFE52D540660082052
:100DAB006A020533020DC2306C0D206B0A206507F9
:100DBB001581158102161722780030640530650203
:100DCB007801E53775F007A4F9E5F028F5F0E9A20D
:100DDB00F013A2F113A2F213F537C39478500375F5
:100DEB003778C3E53795384008D266D292D291D284
:100DFB0090306002A1FC855056855157D26043E676
:100E0B008022207D11C2AF754302C294D295D2AF1E
:100E1B00759F11020FDCC2AF754302C294D293D2FD
:100E2B00AF759F11020FDC307243207D20C2AF756E
:100E3B004303900143757E10D290C293306204C27B
:100E4B0091C150D294D2AF759F01020FDCC2AF7526
:100E5B004303900143757E10D292C295306204C257
:100E6B0091C170D294D2AF759F21020FDC207D17F8
:100E7B00C2AF75430390011ED290306202C291D271
:100E8B00AF759F01020FDCC2AF75430390011ED2F9
:100E9B0092306202C291D2AF759F21020FDC207D8E
:100EAB0011C2AF754304C295D293D2AF759F210285
:100EBB000FDCC2AF754304C293D295D2AF759F01BD
:100ECB00020FDC307243207D20C2AF7543059001C9
:100EDB0032757E20D291C294306204C292C1ECD2A0
:100EEB0095D2AF759F11020FDCC2AF754305900110
:100EFB0054757E08D291C294306204C290E10CD238
:100F0B0093D2AF759F11020FDC207D17C2AF7543D3
:100F1B0005900114D291306202C292D2AF759F112B
:100F2B00020FDCC2AF754305900128D2913062EB02
:100F3B00C290D2AF759F11020FDC207D11C2AF752D
:100F4B004306C293D294D2AF759F01020FDCC2AF9E
:100F5B00754306C295D294D2AF759F21020FDC3038
:100F6B007242207D20C2AF754301900154757E08FB
:100F7B00D292C295306204C290E188D293D2AF75FF
:100F8B009F21020FDCC2AF754301900132757E20A9
:100F9B00D290C293306204C292E1A8D295D2AF75BF
:100FAB009F01E1DC207D16C2AF754301900128D271
:100FBB0092306202C290D2AF759F21E1DCC2AF7555
:100FCB004301900114D290306202C292D2AF759F4E
:100FDB0001C26622900112757E00D292D291D290FC
:100FEB00C295C294C293C2622278807607087607B4
:100FFB000876010876040876FF0876FF08760A085B
:10100B007602087601087601788C7601087600085E
:10101B0076B40876FF0876FF0876FF087603087625
:10102B00FF0876010876FF0876250876D0087678D3
:10103B000876C80876040876FF087601087600085B
:10104B00767A08760A087601087601087600087623
:10105B00FF227887E6FFC272BF0302D2727888C282
:0F106B007DE630E102D27DC27E7889E630E10277
:10107A00D27EC3EF94026008758E01D27302108F7C
:10108A00758E00C273227880E6149000809378A44B
:10109A00F67881E6149000809378A5F67886E614AF
:1010AA0090008D9378A6F6789FE6F8700108C3E859
:1010BA00941140027811E82828F56E256E256E28CD
:1010CA00F56F256E2828F570789CE67538FF753916
:1010DA000CB402067538A075390AB403067538824D
:1010EA0075390578A3E61490009A93F569120FDF13
:1010FA0022227896E6FA7897E6FB7888E6B4030522
:10110A00C3EB940EFB307F047A007BFFC3EB9AFC9F
:10111A00C3948250027C827575000575EC8575F062
:10112A00A4C3E5F0947D40F222D27F11FC1205623D
:10113A007A007B007C10120558E55F2AFA74003B9E
:10114A00FBDCF37C04C3EB13FBEA13FADCF7FEC205
:10115A007F11FC22E5EF20E6037520000520903F71
:10116A00FFE520146006901DFF14600093046003DD
:10117A0075EF1253D9BF7581C043FF8012055375AD
:10118A00EF0243B203E5B3240420E70DF521E5E3BA
:10119A0020E0068521B343E301120FDF7580FF7556
:1011AA00A40075F19075D47F75900775A53F75F207
:1011BA003F75D50075A60175E241E4F8F6D8FD75CC
:1011CA006B01120FF412165F78988676753001C299
:1011DA00AF12056C12057C120562120583120562B4
:1011EA0012058A12056212178212056C12056C1218
:1011FA000567C2AF78FA79FA308707D9FBD8F702C0
:10120A001C00115D119011FB11FC78988676120F63
:10121A00DF75885075891275C82475910475D84090
:10122A0075A82275B80275E690759B80759D007544
:10123A00D10E75BC5875BB0675BA1175E8801205D2
:10124A0053D2AF1208AB53DACF207E0343DA2030F1
:10125A007E0343DA1043DA01C2D8C27112056CD296
:10126A00617B037A0CE55E70077A0CDB030211FCE2
:10127A001205622070030211FCC270E55FC394027A
:10128A0040E1E52F541F856160F561B560D5DAD577
:10129A00C26153DACF207E0343DA20307E0343DA79
:1012AA0010C2D8C27178A2E67008D274E52F54E051
:1012BA00F52FC275752900120567307409C3E5292F
:1012CA00940A4002D27512055878023074027800E6
:1012DA00C3E55F9840F0C2AF12057C12057C120587
:1012EA007CD2AF12056C754D00120558788CE6C396
:1012FA00940150030213C9E530C394015003021349
:10130A00C9207435C3E55F94FF50030213C9C2AF05
:10131A00120591D2AF120567C3E55F940150EFC27F
:10132A00AF12057C12055D12057CD2AF120567C3A8
:10133A00E55F94FF40E90218077F05D27F11FC128E
:10134A000567C2AFC27F11FCAE5FC3E55F947FD26F
:10135A00AF4076120553C2AF120591D2AFDFDC312E
:10136A0033C3EE94057897F612056C1216A112177C
:10137A008A7F0AD27F11FC120567C2AFC27F11FCB5
:10138A00AE5FC3E55F947FD2AF50E6120553C2AF9A
:10139A0012057C12055D12057CD2AFDFD63133EE21
:1013AA0024057896F612056C1216A11217B91205C1
:1013BA006711FCC3E55F94FF5002610B021807C373
:1013CA00E55F954D4003855F4D1205677801798881
:1013DA00E7B403027805C3E55F98400241F3C2AF60
:1013EA00120591120591120591D2AF12056C753052
:1013FA0000E4F531F5320531E531F470390532781A
:10140A009AE67819146012783214600D787D1460A7
:10141A000878FA146003753200C3E532984017154C
:10142A00327531B478998676C2AF120591D2AF7807
:10143A0098867612056712055DE52A7005307402F2
:10144A0021FC78012074027806C3E55F9840A71250
:10145A000567E52A70030211FCC2AF120FDFE4F53B
:0F146A0022F523F524F525F526F56AD2AF78850E
:10147900E6C333F568E4F545F546F547F548F5491A
:10148900F573F52CF52DF53775730875BB10120535
:101499005312093EE5E820ECFBA8BDA9BEE970019D
:1014A900F8887412094275730875BB107887E6FECF
:1014B9007602115D7887EEF6C2AF7564FF1209FDF9
:1014C900852264852265852266D2AF75220175243D
:1014D9000175250175260185636C756D017888E6AE
:1014E900B40307C27D307602D27DD268D2697533E2
:1014F90000120F45120F6A120A1D120A24120A1D40
:10150900120A24120A1D02151EC2AF115DD2AF754F
:10151900730075BB06120CA812065C120DC3120EDD
:101529000D120A24120C97306D031206FC20670372
:1015390012084E306703120895120DC3120E3212AB
:101549000A24120CA8306D03120738120DC3120EAB
:10155900A9120A24120C97306D03120796120DC3B3
:10156900120ECE120A24120CA8306D031207F312C0
:101579000DC3120F45120A2412093E120C97120DBF
:10158900C3120F6A120942120A2430692F206B2CE8
:1015990085676485676585636C756D0179187A0C53
:1015A900C3E533994009C269D26A8A350215C5C3B0
:1015B900E55F9401400302151E02161F306A1B20C5
:1015C9006B18E535147004C26AA112F535C3E55FDD
:1015D9009401400302151E02161F753600C3E56209
:1015E9009401400985676585636C756D01C3E56282
:1015F90078FA985021307404E52A601A78F0306B33
:10160900058567647820C3E541985002A11E053617
:10161900E55F6002C122753600C2AF120FDF78871D
:10162900E6FE7602115D7887EEF6E4F522F523F5FC
:1016390024F525F526F568C268D2AF120553120FB5
:10164900DF307406E52A700221FC788DE6C3940127
:10165900400241D061FB901A0D78201216E3E52073
:10166900B4A50CA31216E3E520B45A03021681129D
:101679000FF41216A10216A0901A0378807B0A12A1
:1016890016E3A308DBF9901A0F788C7B181216E37E
:10169900A308DBF9901A2722C2AF1217221216FCEF
:1016A900901A00740E1216E8A374041216E8A374B3
:1016B900141216E8901A0378807B0A1216E7A30819
:1016C900DBF9901A0F788C7B181216E7A308DBF95F
:1016D900121735121713901A2722E493F622E643BC
:1016E9008F01538FFD75EF0275B7A575B7F1F053EB
:1016F9008FFE22438F02438F0175EF0275B7A575DF
:10170900B7F1901A0DF0538FFC22901A0D74A5D1E0
:10171900E8901A0E745AD1E8227A3079D07820905C
:101729001A40D1E3E520F709A3DAF7227A3079D014
:10173900901A40E7D1E809A3DAF922AB77A878BB78
:1017490001027980BB02027981BB03027982BB0461
:10175900027994BB05027983BB06027986BB07022D
:101769007992BB08027987BB0902799CBB0A027985
:1017790088BB0B027989E8F7227C0512056CDCFB32
:1017890022C2AF12057C12058312058A1205911235
:10179900055D12057C12058312058A120591120551
:1017A9005D12057C12058312058A120591D2AF22BA
:1017B900C2AF12059112058A12058312057C120522
:1017C9005D12059112058A12058312057C12055DC9
:1017D90012059112058A12058312057CD2AF22AE39
:1017E90077AF78C2AF12057C12057C12057C120511
:1017F9005DDEF212059112055DDFF8D2AF221217F4
:101809008A12178212178275770175780175790026
:101819001217E87C05AD5F12056CC3ED955F70F595
:10182900C3E55F9401400AC3E55F94FF403702189E
:101839004B1217441216A112178AC2AF75EF121272
:101849001782DCD10579C3E5799403500280C1126E
:1018590017820578E5771490009F93F808C3E57817
:0E18690098500280A81217821217820577C3CA
:10187700E577940C50028094120FF41216A1C2AFB0
:0618870075EF121217823A
:0319FD0002115E76
:101A00000E041407070104FFFF0A020101A55A0191
:101A100000B4FFFFFF03FF01FF25D078C804FF01DA
:081A200000FF0A010100FFFFB5
:101A400023454D41583430412320202020202020A0
:101A500023424C48454C4923463333302320202031
:101A60002020202020202020202020202020202076
:101C0000C2AFC2D353D9BF7581C043B20343FF8073
:101C1000752438752503B1C975EF0275E24043F1AB
:101C20008053A47F75D400D2877DFA780379E67C4F
:101C300010752200752300901DD67B0675249875BB
:101C400025013087028142208708D8FBD9F9DCF7CB
:101C500081B4308708D8FBD9F9DCF781B4B189E4C5
:101C600093A3C39A6004DDC381B4DBDBB17B600264
:101C7000812B7B08E493FAA3B15CDBF87A30B15C8A
:101C8000752200752300B17BEAFCEBFDC3ED94FEE9
:101C9000400EB17B8A278B28ED30E0048A828B834B
:101CA000B17B7AC270D8C3ED94FE601350CEBD00F4
:101CB00025EC60097520007521FF0200008100A855
:101CC00027A9280809D804D90281D3B17FEA89AAB3
:101CD000F281C50D81A0C3ED94035049EDA2E092BD
:101CE000007AC5C3E5829400E583941C50902000DF
:101CF00010438F02438F0175B7A575B7F1F030001F
:101D00001FA827A9280809438F01538FFDD804D99C
:101D100002A12089AAE275B7A575B7F1F0A3A10DBC
:101D2000538FFC817C7AC1BD030CE493A3FAB140CC
:101D3000DCF8B138817C817EAA22AB23B15CEBFA5E
:101D4000EA6222752608C3E52313F523E52213F57D
:101D50002250066323A0632201D526EAB1C9B1C986
:101D600075260AEAF4200102D287300102C287B147
:101D7000C9C3134002C201D526EB22B17FEAFB2082
:101D80008702A17F308702A184752608AE24AF2583
:101D9000C3EF13FFEE13FEB1CDB1C9C3EA13308711
:101DA000024480FA30E703632201C3E52313F523DD
:101DB000E52213F52250066323A0632201D526D91C
:101DC000E52265236523F52222AE24AF250E0FDE22
:101DD000FEDFFCD20122424C48656C693437316326
:041DE000F3300601D5
:00000001FF
